:020000040000FA
:040000006028423002
:08000800A000030EA100831209
:100010008B1C36288B1031181328B11C36286430FD
:100020000102031C35280000000000000000000051
:1000300000000000000000000000000000000000C0
:100040000000000000003110B114A81003100519C1
:100050000314AA0DA90DA80DB00B362831152A08D6
:10006000AF002908AE002808AD00B11081010B11C6
:0A007000210E8300A00E200E0900EF
:1000C000203084008001840A80300402031C6228EE
:1000D0001230B0001A228501870183160C30850585
:1000E000870183128316051487150716831285016D
:1000F00087010730990000309A00103083168E0077
:100100008312603083168F008312003083169100B3
:100110009F008312C8308316810083123130900013
:10012000003083168C00831210308B008316003051
:100130009B001C141A088312BD00851D002783161E
:1001400010309B001C141A088312BE005E2281012D
:100150008E018F010B118B100B108C018B17BE20A1
:100160003119D420B30BBC28031085190314BA0D20
:10017000F0303A0203196221C023AF28640031181D
:1001800008000B1D08000B11B11031141230B00023
:10019000051DCF2832148316011383120800321074
:1001A0008316011783120800321CDB282D0903393E
:1001B000AD00AE09AF09E4302F02F0300319AF00F3
:1001C0004C302F020C300319AF006C302F023C3042
:1001D0000319AF00EC302F02FC300319AF00B3302D
:1001E0002F02F3300319AF001B302F020F30031919
:1001F000AF003B302F023F300319AF00BB302F025E
:10020000FF300319AF0031110130B7008B132030DC
:10021000370783169B001C141A088312A400A5003C
:1002200025101030370783169B001C141A08831200
:10023000A3000030370783169B001C141A08831292
:10024000A2008B1722082D02031D5C2923082E060D
:10025000FC39031D5C29AF13AF12AF11AF10240896
:100260002F02031D452901303702031D3C293E188A
:100270003C293E143F144E2202303702031D45290B
:10028000BE184529BE143F14522225082F02031D13
:100290005C2901303702031D52293E1C52293E10B1
:1002A0003F14562202303702031D5B29BE1C5B2916
:1002B000BE103F145A225C29B70A033037020318D4
:1002C000080006293D1C0800B601B3019630B400B1
:1002D0000130B5000130B70085018701B113D1218C
:1002E000BE20B30B8929031085190314BA0DF03011
:1002F0003A020319C129B41F0710B40B8929370822
:10030000B6080319B600031987290714B6039630F7
:10031000B400311D70293111321C93292D09033984
:10032000AD00AE09AF0951302F0655390319A82980
:1003300005302F0655390319A82915302F065539D0
:100340000319A82955302F0655390319A8297029F2
:10035000AF13AF12AF11AF108B1320303707BC00B3
:100360002F08BB00052210303707BC002E08BB0049
:10037000052200303707BC002D08BB0005228B1773
:10038000CB2185018701B70AB60103303702031C70
:1003900070295E2208000230370203190800850127
:1003A00087016430B90001300F1E87000F1A8701E2
:1003B000BE20311DD3293111321CE3292D09033907
:1003C000AD00AE09AF0951302F0655390319D129B7
:1003D00005302F0655390319D12915302F06553907
:1003E0000319D12955302F0655390319D129B90BD5
:1003F000D3298501870108003F1C08003F101030F9
:10040000BC003E08BB00052208008B133B08831686
:100410001C159A0083123C0883169B0055309D00E2
:10042000AA309D009C1464009C18132A1C1183128E
:100430008B17080000309500603084008B13831602
:1004400004089B001C141A0883128B178000840A6E
:1004500068300402031C1E2A6430D5002D24DC0001
:100460003C30EC00ED00EE00EF00EA146E30D500F9
:100470002D240F39031D080032240F39031D0800F5
:1004800037240F39031D08003C240F39031D0800D1
:100490008316871107128312EA1008000130E80062
:1004A0006D2208000430E8006D2208000230E800E8
:1004B0006D2208000830E8006D220800EA178B134F
:1004C000831670309B001C141A0883128B17E800E7
:1004D0006D220430EB00EA130800E8080319080055
:1004E000681C7A2A6730D5002D24D1006830D500E9
:1004F0002D24D200E81C842A6730D5003224D10094
:100500006830D5003224D200681D8E2A6730D500AD
:100510003724D1006830D5003724D200E81D982A4E
:100520006730D5003C24D1006830D5003C24D2008F
:10053000681EA22A6A30D5002D24D1006B30D50068
:100540002D24D200E81EAC2A6A30D5003224D10016
:100550006B30D5003224D200681FB62A6A30D5002D
:100560003724D1006B30D5003724D200E81FC02AD1
:100570006A30D5003C24D1006B30D5003C24D20039
:10058000EA16D11AD02A511BD02A511CD02ADC1FBE
:10059000EA125C1FD02A501CD02AC01BD02A0800A7
:1005A000EA1EE02AEA1BE02A511870308B138316EA
:1005B0009B001C141A0883128B1768020319080089
:1005C000D11AEB2A511BEB2A6A10511CEB2A50144A
:1005D000051E6A140516511CF32A511A5016D11A19
:1005E000C017511B5012EA1FFA2AD11A0800511BDA
:1005F0000800FE2AD11A2B2B511B2B2B6530D5005E
:10060000521A2D24D21A3224521B3724D21B3C24D6
:100610005118C4006630D500521A2D24D21A322443
:10062000521B3724D21B3C245118CC0052085118BD
:10063000D70004306A183230EA1B32305118C80033
:1006400051185C14EA1F292B511C282B4403C000AD
:1006500008005118C00151187030BC006808E9004A
:10066000BB000522BE010800FD010730FF007B082A
:10067000FE0C03183F2BFF0B382BFB01003403103B
:10068000442BFE0C0318FB07FB0CFD0CFF0B412B4E
:10069000FB0CFD0C003494019301093095008B1381
:1006A0008E018F018B17D6135608FB007508F51BBA
:1006B000FF3CFE00FE133423FD0D7B0DF51FD60716
:1006C000F51BD60256087607930003181414083059
:0406D0009500080089
:1007800002300F02031C0800EA1CDD2BA127F10830
:100790000319DD2B6E30D50071182D24F118322489
:1007A00071193724F1193C24E80068184E22E81822
:1007B000562268195222E8195A220730EB050330F5
:1007C0008A006B088207E82B182C192C1A2C1B2C7A
:1007D000501C262C4008D500571A2D24D71A322435
:1007E000571B3724D71B3C24D6006108F50060084E
:1007F000F6005C1C4B23C80B262C4C085C180530FB
:10080000C8005C1CC00A5C1044084002031C262C73
:10081000C01B0E2C501E0E2CC001262C5012DC18B2
:1008200005125C1950105C1DC0035C1DC017262CFE
:10083000262C262C262C071C1F2C0710262CE908FA
:100840000319262C07140310E90C262CEB0A05309B
:100850006B020318EB018F01080005308A00D513E5
:100860005508820005308A00D517550882000630E9
:100870008A00D5135508820006308A00D51755081E
:020880008200F4
:100A000080340134033404340534063408340934A2
:100A10000A340B340D340E340F34113412341334C1
:100A2000143416341734183419341B341C341D3460
:100A30001E342034213422342434253426342734FF
:100A400029342A342B342C342E342F34303432349D
:100A50003334343435343734383439343A343C343C
:100A60003D343E34403441344234433445344634DA
:100A7000473448344A344B344C344D344F3450347A
:100A800051345334543455345634583459345A3418
:100A90005B345D345E345F346134623463346434B7
:100AA00066346734683469346B346C346D346E3456
:100AB00070347134723474347534763477347934F4
:100AC0007A347B347C347E34C4346434013401346D
:100AD0001134003401341134003400340034003453
:100AE0000034003400340034003400340034003466
:100AF0000034003400340034003400340034003456
:100B0000FF347E347C347B347A34793477347634F1
:100B1000753474347234713470346E346D346C34B2
:100B20006B346934683467346634643463346234F3
:100B300061345F345E345D345B345A345934583434
:100B40005634553454345334513450344F344D3476
:100B50004C344B344A3448344734463445344334B7
:100B6000423441343F343E343D343C343A343934F9
:100B700038343734353434343334323430342F3439
:100B80002E342C342B342A3429342734263425347B
:100B900024342234213420341E341D341C341B34BC
:100BA00019341834173416341434133412341134FD
:100BB0000F340E340D340B340A340934083406343F
:100BC0000534043403340134C4346434013401344E
:100BD0002234003401342234003400340034003430
:100BE0000034003400340034003400340034003465
:100BF0000034003400340034003400340034003455
:100C000080340034003401340234033404340634B4
:100C100008340A340C340E341134143417341A34B2
:100C20001D342134243428342C342F3433343734D5
:100C30003B343F34433447344B344F3452345634CE
:100C40005A345D346134643467346A346D347034DA
:100C500072347434763478347A347B347C347D3432
:100C60007E347E347E347E347E347D347C347B34FA
:100C70007A34783476347434723470346D346A343F
:100C80006734643461345D345A34563452344F34EA
:100C90004B34473443343F343B34373433342F34CC
:100CA0002C342834243421341D341A3417341434A9
:100CB00011340E340C340A3408340634043403344A
:100CC0000234013400340034C43464340134113447
:100CD00044340034013444340034003400340034EB
:100CE0000034003400340034003400340034003464
:100CF0000034003400340034003400340034003454
:100D000080340034003401340234033404340634B3
:100D100008340A340C340E341134143417341A34B1
:100D20001D342134243428342C342F3433343734D4
:100D30003B343F34433447344B344F3452345634CD
:100D40005A345D346134643467346A346D347034D9
:100D500072347434763478347A347B347C347D3431
:100D60007E347E347E347E347E347D347C347B34F9
:100D70007A34783476347434723470346D346A343E
:100D80006734643461345D345A34563452344F34E9
:100D90004B34473443343F343B34373433342F34CB
:100DA0002C342834243421341D341A3417341434A8
:100DB00011340E340C340A34083406340434033449
:100DC0000234013400340034C43464340134413416
:100DD0008834003401348834003400340034003462
:100DE0000034003400340034003400340034003463
:100DF0000034003400340034003400340034003453
:100E00003D1C08006C146D14EB011430B600071083
:100E10000130EB0507308A006B088207102F172F6F
:100E20006108F5006008F6000516D6011A2F7F301C
:100E3000D6001A2F701A432F6B18232F7019F60A39
:100E40007018F603272F7019F50A7018F503503043
:100E50007018EC007019ED00C8307602C830031825
:100E6000F600503076025030031CF600F51F3E2F7E
:100E7000A0307502A030031CF500432F64307502CA
:100E800064300318F5007F30D6006B1CD6014B236D
:100E9000EA017927701C4E2F6D1B7016701D522FA2
:100EA0006C1B7016701E572FEB0A6B1C682F0710F7
:100EB000B60B5F2F07143C306B180A30B600640085
:100EC0000A300F02031C5F2F8F01701A082F1A2F90
:100ED0007508E1007608E000603084000408BC007A
:100EE0000008BB000522840A68300402031C6E2F30
:100EF0000800F0010A30851DEC078519EC027830F6
:100F00006C020319701479300318EC0015306C0270
:100F10000319F0141430031CEC000A30051CED0713
:100F20000518ED0278306D02031970157930031839
:100F3000ED0015306D020319F0151430031CED009F
:100F40000800F1010A30871DEE0702308719EE0212
:100F500078306E020319711479300318EE001530E1
:100F60006E020319F1141430031CEE000A30071E40
:100F7000EF070230071AEF0278306F02031971157C
:100F800079300318EF0015306F020319F115143092
:060F9000031CEF00080045
:084000000C00000004000500A3
:02400E00CC33B1
:10420000010003000300030003000200020002009B
:10421000020000000000FF00FF00FF00FF00FF00A1
:10422000000000000000000000000000000000008E
:104230000000C000C000FF00FF00FF00FF00FF0003
:104240000100510005001500550051000500150042
:10425000550051000500FF00FF00FF00FF00FF00B8
:10426000FF00FF00FF00FF00FF00FF00FF00FF0056
:10427000FF00FF00FF00FF00FF00FF00FF00FF0046
:10428000FF00FF00FF00FF00FF00FF00FF00FF0036
:10429000FF00FF00FF00FF00FF00FF00FF00FF0026
:1042A000FF00FF00FF00FF00FF00FF00FF00FF0016
:1042B000FF00FF00FF00FF00FF00FF00FF00FF0006
:1042C0007D00FC007D00FC007D00FC007D00FC000A
:1042D000FF00FF00FF00FF00FF00FF00FF00FF00E6
:1042E0000000000000000000FF00FF00FF00FF00D2
:1042F000FF00FF00FF00FF00FF00FF00FF00AA001B
:00000001FF
